:020000040800F2
:10000000001800205B5B0008095B0008D15B00085A
:100010000D5B00080F5B0008115B0008000000008A
:10002000000000000000000000000000135B00085A
:10003000155B000800000000175B00085D0E00085B
:100040001B5B00081D5B00081F5B0008215B0008AC
:10005000235B0008255B0008275B0008295B00087C
:100060002B5B00082D5B00082F5B0008315B00084C
:10007000335B0008355B0008375B0008395B00081C
:100080003B5B00083D5B00083F5B0008415B0008EC
:10009000435B0008455B0008475B0008495B0008BC
:1000A0004B5B00084D5B00084F5B0008D10E000859
:1000B000535B0008555B0008575B0008595B00085C
:1000C00082B0002301930093304A116880235B02C1
:1000D0000B431360110080229202A020C0010B6824
:1000E00013400093019B01330193009B002B02D12D
:1000F000019B8342F3D1254B1B689B0339D5244BCD
:1001000011221A60214A5368F0218B435360214B1E
:100110001B68102B2FD0042B32D01C4B5A685A600E
:100120001A4B5A685A605A681B490A405A60596803
:10013000882252030A435A601968802252040A43F3
:100140001A601900802292040B681342FCD00F4BF6
:100150005A6803218A435A605A6801390A435A602F
:1001600019000C224B681340082BFBD1074B0122CE
:100170001A6302B07047536840390B435360CFE7AE
:10018000024A536890210B435360C9E700100240B4
:0C01900000200240DC140020FF7FC0FFB4
:10019C00124B1B68002B0FD1104B32221A60104BE4
:1001AC001B68012B0ED90F4B1B68002B05D0013B94
:1001BC000C4A1360002B00D070470B4B802252006E
:1001CC009A61F9E7002B04D1074B802252049A6103
:1001DC00F2E7054B802252009A61EDE750150020A2
:0C01EC00581500205C150020000400489D
:1001F80010B5054B1860002805D01C00FFF7CAFF92
:0C0208002368002BFAD110BD6015002007
:1002140010B504F06DFC154B1A68D34301321BD0A2
:10022400FF22110019401A4217D0114A11601B0213
:100234001B0E16D00F4A13600E4B1A680E4B1A6031
:100244000E4B1968CA43FF23180088430C49086001
:10025400120C13400B4A136010BD054A0B211160A8
:10026400E5E7044B0A221A60E6E7C046006400088A
:1002740068150020FC140020C81400200464000841
:0802840054150020581500205C
:10028C0010B544490122CB681A42FCD1414B1B6981
:10029C001B0604D53F4B404A5A60404A5A603D4BBE
:1002AC001A6902210A431A613D4A5A611A693E31A0
:1002BC000A431A6119000122CB681A42FCD1354B52
:1002CC00DB689B0604D5334AD36820210B43D360EB
:1002DC00304B1A6902218A431A611A6901390A439F
:1002EC001A61304B1B68DB432D4A138029490122CC
:1002FC00CB681A42FCD1274BDB689B0604D5254AF8
:10030C00D36820210B43D360274B1B68DB43274A60
:10031C00138020490122CB681A42FCD11D4BDB68AB
:10032C009B0604D51B4AD36820210B43D360204B7A
:10033C001B68DB431F4A138016490122CB681A4203
:10034C00FCD1144BDB689B0604D5124AD3682021E0
:10035C000B43D360184B1B68DB43184A13800D49C1
:10036C000122CB681A42FCD10A4BDB689B0604D5F0
:10037C00084AD36820210B43D360064B1A6901212C
:10038C008A431A611A697F310A431A610A20FFF7FE
:10039C002DFF10BD0020024023016745AB89EFCD36
:1003AC000064000868150020FC140020026400089A
:1003BC005415002004640008581500200664000839
:1003CC00F8B5C54B1C68631E012B00D91BE2C34951
:1003DC000122CB681A42FCD1C04B1B691B0604D509
:1003EC00BE4BBF4A5A60BF4A5A60BC4A13690221CD
:1003FC000B431361012C00D1C8E0B84BBA4A5A61C7
:10040C00B64A136940210B43136111000122CB68DA
:10041C001A42FCD1B14BDB689B0604D5AF4AD368BA
:10042C0020210B43D360AD4B1A6902218A431A6118
:10043C001A6901390A431A61013C63425C41644206
:10044C00AA4B1C40A84B9C466444A94B1B68013327
:10045C00DB432380A1490122CB681A42FCD19F4B7C
:10046C00DB689B0604D59D4AD36820210B43D360DF
:10047C00A04B1B68DB43638098490122CB681A426E
:10048C00FCD1964BDB689B0604D5944AD36820219B
:10049C000B43D360984B1B68DB43A3808F4901222D
:1004AC00CB681A42FCD18D4BDB689B0604D58B4A7A
:1004BC00D36820210B43D360904B1B68DB43E38054
:1004CC0086490122CB681A42FCD1844BDB689B061F
:1004DC0004D5824AD36820210B43D360884B1B6818
:1004EC001B02884A12781343DB4323817B49012288
:1004FC00CB681A42FCD1794BDB689B0604D5774A52
:10050C00D36820210B43D3607F4B1B68DB43638193
:10051C0072490122CB681A42FCD1704BDB689B06F6
:10052C0004D56E4AD36820210B43D360774B1B68EC
:10053C001B061B0C764A12781343DB43A3816749D5
:10054C000122CB681A42FCD1644BDB689B0604D5B4
:10055C00624AD36820210B43D3606E4B1B68DB438C
:10056C00E3815E490122CB681A42FCD15B4BDB680C
:10057C009B0604D5594AD36820210B43D360103411
:10058C006548564B01222025644E07E01300644A4F
:10059C005A6135E704340430B04219D00168C943BC
:1005AC002180D9680A42FCD1D9680D4202D0D968A1
:1005BC002943D9600168C943090C6180D9680A4292
:1005CC00FCD1D9680D42E5D0D9682943D960E1E75F
:1005DC00424B1A6901218A431A611A6901310A4393
:1005EC001A613D4B1C68012C2DD03C4B4D4A5A6175
:1005FC003A4A136940210B43136111000122CB6865
:10060C001A42FCD1354BDB689B0604D5334AD368C0
:10061C0020210B43D360314B1A6902218A431A61A2
:10062C001A6901390A431A61013C63425C41644214
:10063C002E4F27403B4B9C4667443C00274B0122E6
:10064C002025394E07E0254B384A5A61D0E704344F
:10065C000430B04219D00168C9432180D9680A42DC
:10066C00FCD1D9680D4202D0D9682943D960016800
:10067C00C943090C6180D9680A42FCD1D9680D4282
:10068C00E5D0D9682943D960E1E780239B009C46DB
:10069C0067442748114B01222025264E03E00437DE
:1006AC000430B04248D00168C9433980D9680A4245
:1006BC00FCD1D9680D4202D0D9682943D960418850
:1006CC00C9437980D9680A42FCD1D9680D42E6D079
:1006DC00D9682943D960E2E7541500200020024074
:1006EC0023016745AB89EFCD0074000800F4FFFFD0
:1006FC0058150020FC14002040150020DC140020AC
:10070C00D0140020D8140020D4140020F814002099
:10071C00F41400203015002004080020F40B0020F5
:10072C000068000800780008F40D0020006C000838
:10073C000402002004040020334B1A6901218A436F
:10074C001A611A6901310A431A61304B1C68012C79
:10075C002CD02D4B2E4A5A612B4A136940210B4346
:10076C00136111000122CB681A42FCD1264BDB68C5
:10077C009B0604D5244AD36820210B43D360224B1B
:10078C001A6902218A431A611A6901390A431A61EA
:10079C00013C63425C4164421E4B1C401C4B9C461A
:1007AC006444194B012220251B4E07E0164B1B4AB3
:1007BC005A61D1E704340430B04218D00168C943FF
:1007CC002180D9680A42FCD1D9680D4202D0D9687F
:1007DC002943D9604188C9436180D9680A42FCD158
:1007EC00D9680D42E6D0D9682943D960E2E7064BB7
:1007FC001A6901218A431A611A697F310A431A6105
:10080C000A20FFF7F3FCF8BD00200240541500202D
:10081C00007C000800F4FFFF0408002000700008B2
:10082C00284A91698023DB010B4393619023DB05FC
:10083C001A6825490A401A601968A02292030A43D3
:10084C001A605A6A21490A405A62596A882252002F
:10085C000A435A621E4B1F4A13601F4A13601F4BF8
:10086C001B68392B29D01ED8132B28D0263B5A1E97
:10087C0093415B421A4A13401A4A944663441A4AFB
:10088C00938180239B025360002393602C3313606D
:10089C00136801210B431360144B1960144B802215
:1008AC0012051A607047603B5A1E93415B42114A15
:1008BC001340114A94466344E1E7104BDFE7104BB9
:1008CC00DDE7C04600100240FFFFEBFF0FF0FFFF1B
:1008DC001411002048150020441500206815002034
:1008EC00BFFCFFFFE204000000380140641500204B
:1008FC0000E100E019EEFFFF881300004103000047
:04090C00C40900001A
:100910000A498022CB691A42FCD080B2074B188565
:10092000074B1B68032B00D07047064B80225204F4
:100930009A61054B04221A60F6E7C0460038014070
:0C09400058150020000400485C15002041
:10094C00F0B5C64600B54F4B1B68002B66D0013B7B
:10095C005A4253415B424C4C1C404C4B9C466444A9
:10096C002068C3436168CA430140013100D16FE084
:10097C001904090C0139464801601B0CFF210B407E
:10098C004448036044480360130C0B4043490B601C
:10099C00012B04D0102B02D00B0001211960120482
:1009AC00120C3F4B1A60A368DB439A05920F3D492A
:1009BC000A603F221A403C490A601B0C3B4A1360F8
:1009CC00E368DB439846250010351E0C384B1E603F
:1009DC003601324B1F683900300005F071FB354B86
:1009EC00186043461B041B0E7E2B01D901235B426E
:1009FC00314A1360BE422ED2304A314908CDDB4316
:100A0C0008C28A42FAD1C023DB009C4664442D4ABA
:100A1C002D4808CCDB4308C28242FAD103F09AFE7F
:100A2C001F4B1B68002B07D09023DB051B8A5B0533
:100A3C0002D41B4B00221A600D20FFF763FF01F05C
:100A4C00D1F9174B1B68002B15D180BCB846F0BDF3
:100A5C0004F04AF8E2E702F093FA02F02BFBFF23D2
:100A6C00424613407E2B01D901235B42174A136087
:100A7C0002F07AFBC0E7013B154A136003F076FBEA
:100A8C00E3E7C0465415002000F4FFFF0074000893
:100A9C0058150020FC140020C8140020DC14002081
:100AAC0040150020D0140020D8140020D4140020AD
:100ABC003015002014150020F81400200408002024
:100ACC00F40D00200402002004080020F41400207F
:040ADC00F0140020F2
:100AE00070B5041E00DA9CE0092C00D893E0632C5A
:100AF00000D881E0FA239B009C426ED3534B9C426A
:100B00005AD9534B9C4248D9524B9C4236D9524BEE
:100B10009C4224D9514B9C4212D9514B9C4200D942
:100B200084E05049200005F0D1FA05004D4920002D
:100B300005F0F1F90C0028003030C0B2FFF7E8FEF4
:100B40004949200005F0C2FA05004749200005F098
:100B5000E2F90C0028003030C0B2FFF7D9FE43495B
:100B6000200005F0B3FA05004049200005F0D3F954
:100B70000C0028003030C0B2FFF7CAFE3C4920000C
:100B800005F0A4FA05003A49200005F0C4F90C006C
:100B900028003030C0B2FFF7BBFE3649200005F018
:100BA00095FA05003349200005F0B5F90C0028003E
:100BB0003030C0B2FFF7ACFEFA218900200005F00A
:100BC00085FA0500FA218900200005F0A4F90C003F
:100BD00028003030C0B2FFF79BFE6421200005F0F2
:100BE00075FA05006421200005F095F90C00280035
:100BF0003030C0B2FFF78CFE0A21200005F066FA03
:100C000005000A21200005F086F90C00280030308C
:100C1000C0B2FFF77DFE20003030C0B2FFF778FE93
:100C200070BD2D20FFF774FE64425DE7124920007D
:100C300005F04CFA05001049200005F06CF90C0095
:100C400028003030C0B2FFF763FE6AE70F270000CC
:100C50009F8601003F420F007F969800FFE0F50558
:100C6000FFC99A3B00E1F5058096980040420F00CD
:0C0C7000A08601001027000000CA9A3B7B
:100C7C0070B5484D484C02E06420FFF7B7FA474B7B
:100C8C005969802292020A435A6159698022D20220
:100C9C000A435A619021C90500260E60404B1E6024
:100CAC00404ACA60DA60D9683F480140D9601A6886
:100CBC0002401A601968802252020A431A6080228C
:100CCC0052009A6101232B60FFF7F4F9374B1E6039
:100CDC00374B1E60374B1E60374B0B221A60374B5D
:100CEC001E600A23364A1360364A1360364B0322C1
:100CFC001A60364B364A1A602B685901C91A89009A
:100D0C00C918C900334B186805F0DAF9013880238B
:100D1C005B0498420DD2304A50603048036A1B0283
:100D2C001B0AC02109060B4303620023936007339F
:100D3C0013603220FFF75AFA03F00CFDFFF764FA48
:100D4C000220FFF753FAFFF76BFD0220FFF74EFA74
:100D5C000D20FFF7D7FD224804F077FF3120FFF775
:100D6C00D1FD2E20FFF7CEFD0B20FFF7B3FE1D4863
:100D7C0004F06BFFFFF7E4FD03F054FD01F0AEFB54
:100D8C00002800D178E72368002BF5D003F052FA45
:100D9C00F2E7C046DC140020BC1400200010024016
:100DAC0000040048AAAAAAAAFFFFFCFF5C150020B9
:100DBC00601500204C1500206815002064150020DB
:100DCC00FC140020C814002058150020E414002046
:100DDC00A1B0B9120002002010E000E000ED00E02C
:080DEC00EC5B00086C540008E8
:100DF40010B5FFF7D1F9114B1B68114A12689342E1
:100E040019D05A1C0D490A601B788020000218432F
:100E14000C4B1B689A420BD00B4B1B68012B06D959
:100E24000A4B802252049A61094B04221A6010BDB5
:100E3400084A0A60F0E70020F9E7C046441500209C
:100E440048150020FC01002058150020000400482B
:080E54005C15002014110020C0
:100E5C00164B1B68002B02D0013B144A1360144B39
:100E6C001B68002B02D0013B114A1360114B1B680D
:100E7C00002B02D0013B0F4A13600F4B1B68002B59
:100E8C0002D0013B0C4A13600C4B1B68002B02D0A8
:100E9C00013B0A4A13600A490A6853035A40530C2F
:100EAC0053405A0153400B607047C0465015002008
:100EBC00601500204C15002008150020CC140020D3
:040ECC00E41400200A
:100ED00010B5114BDB699B0612D50F4B9B8C99B259
:100EE000FF221340022B0CD0042B12D00B4A1368A4
:100EF0001970136801331360094A1268934204D0D1
:100F000010BD084BFD3A1A60F0E7044B064A1A6020
:100F1000F6E700F095FDF3E70038014048150020A2
:0C0F2000FC010020C0140020141100206F
:100F2C00024A202311680B43136070471C150020E4
:100F3C00064A1368043B1360054A0C32934204D2F0
:100F4C00044A042311680B4313607047E01400201B
:080F5C00881300201C15002081
:100F6400084B1A68111D1960074B6033994202D26D
:100F7400136853607047054A042311680B431360D8
:100F8400F8E7C046E0140020881300201C15002058
:100F9400044B19680A1F1068096811601B681860FF
:080FA4007047C046E014002074
:100FAC00034A1368191D11601A1F12685A607047A2
:040FBC00E01400201D
:100FC000074A1368190008390868043B1B680B605E
:100FD0001368191F1B680B60136818607047C046C0
:040FE000E0140020F9
:100FE400074A13681968181F006818601368181FE7
:100FF400083B1B6803601368083B19607047C046D0
:04100400E0140020D4
:101008000C4B19680A680C4BCB1A9B109B1A042BC3
:1010180006D4002A0AD092008A1A13680B60704717
:10102800064A042311680B431360F8E70439014B9F
:101038001960F4E7E0140020881300201C15002034
:1010480030B5144B1A681168134BD31A9B105B1AEE
:10105800042B19D4043A0F4B1A60012913D9012320
:101068005B1A9B009D580222521A9200094C236871
:1010780098589B18043B1860013904320029F6D1AE
:10108800044B1B681D6030BD044A042311680B43E0
:101098001360F8E7E0140020881300201C150020D6
:1010A800F0B5144B1A681568134BD31A9B105B1BC9
:1010B800042B19D4043A17680E4B1A60012D12D963
:1010C8006E1E0422524200211C00236898589B1867
:1010D80058600131043AB142F7D101235D1B054B39
:1010E8001B68AD00EF50F0BD044A042311680B43A0
:1010F8001360F8E7E0140020881300201C15002076
:10110800054B1A68111F12680868844662440A6011
:0C1118001A68043A1A607047E0140020C6
:10112400024B1A681368013313607047E0140020FF
:10113400054B1A68111F12680868821A0A601A6837
:0C114400043A1A607047C046E014002016
:10115000024B1A681368013B13607047E0140020CB
:10116000044B1A681368002B00DB70475B42136066
:08117000FBE7C046E01400207B
:1011780010B50F4B1B681A68D117501848401F2824
:1011880009DC191F0A4C2160002A0BDB0B000968D7
:101198009140196010BD074A8023DB0011680B439A
:1011A8001360F7E7043B1A68C2401A60F2E7C046CA
:0811B800E01400201C150020CA
:1011C000054B1A68111F1268086802400A601A6805
:0C11D000043A1A607047C046E01400208A
:1011DC00054B1A68111F1268086802430A601A68E6
:0C11EC00043A1A607047C046E01400206E
:1011F800054B1A68111F1268086842400A601A688D
:0C120800043A1A607047C046E014002051
:10121400024B1A681368DB4313607047E014002024
:10122400024B1A6813685B4213607047E014002095
:10123400054B1A68111F1268086842430A601A684D
:0C124400043A1A607047C046E014002015
:1012500010B50B4B1C682168002909D0043C20689C
:1012600004F016FF2060064A1368043B136010BDAB
:10127000044A80231B0111680B431360F7E7C04643
:08128000E01400201C15002001
:1012880010B50B4B1C68216800290AD0221F106872
:10129800083C23685843064B1C6004F0F5FE2060A8
:1012A80010BD044A80231B0111680B431360F7E744
:0812B800E01400201C150020C9
:1012C00010B50B4B1C682168002909D0043C20682C
:1012D00004F010FF2160064A1368043B136010BD40
:1012E000044A80231B0111680B431360F7E7C046D3
:0812F000E01400201C15002091
:1012F80070B50D4B1C682568002D0ED0043C26687F
:101308002900300004F0F2FE2160074B1C68290018
:10131800300004F0B9FE206070BD044A80231B0130
:1013280011680B431360F7E7E01400201C15002038
:101338000B4B1B681A681F2A0BD8043B01219140EC
:101348000A0019680A431A60054A1368043B1360C7
:101358007047044A8023DB0011680B431360F7E7EA
:08136800E01400201C15002018
:101370000B4B1B681A681F2A0AD8043B01219140B5
:101380001A688A431A60064A1368043B1360704760
:10139000044A8023DB0011680B431360F7E7C04663
:0813A000E01400201C150020E0
:1013A8000C4B1B681A681F2A09D8012191400A00B2
:1013B800191F0968114209D001221A6005E0064A7E
:1013C8008023DB0011680B431360704700221A600A
:0C13D800FBE7C046E01400201C150020BC
:1013E400034A1368191D1160024A12685A60704753
:0813F400E0140020E4140020C5
:1013FC00064A1368191F1B6808681B1A5842434198
:10140C000B601368043B13607047C046E014002067
:10141C00064A1368191F1B6808681B1A581E83415B
:10142C000B601368043B13607047C046E014002047
:10143C00034B1A6811684B424B4113607047C0460E
:04144C00E014002088
:10145000074B1A68131F012112681868904200DCBC
:1014600000211960024A1368043B13607047C046AC
:04147000E014002064
:1014740030B5074B1A68111F10680A68D217C40FD9
:101484000D68854262410A601A68043A1A6030BDE8
:04149400E014002040
:10149800074B1A68131F012112681868904200DB75
:1014A80000211960024A1368043B13607047C04664
:0414B800E01400201C
:1014BC00064A1368191F1B68086884469C459B41A3
:1014CC005B420B601368043B13607047E014002010
:1014DC0030B5074B1A68111F08681468C20FE5175E
:1014EC0084426A410A601A68043A1A6030BDC046E8
:0414FC00E0140020D8
:10150000114B1A681368002B0CD0C82B0ADC190089
:10151000C83107DB002B0CDD013B9B000B495B58FE
:10152000136005E00A4A8023DB0011680B43136057
:101530007047DB439B00111F086804495850083A64
:10154000014B1A60F4E7C046E0140020F40D0020BF
:041550001C15002046
:10155400044B0A221A60044B1B68002B01D1034B75
:101564001A607047C814002020150020FC140020C5
:10157400044B10221A60044B1B68002B01D1034B4F
:101584001A607047C814002020150020FC140020A5
:1015940005490A681368043A0A60002B02D0013B2B
:0C15A400002BFCD17047C046E014002072
:1015B00004490B6864221868424303480260043BF4
:0C15C0000B607047E0140020CC140020E9
:1015CC0010B5054B1C68221D1A60044B1868642169
:1015DC0004F076FD606010BDE0140020CC140020F7
:1015EC0030B5094B1B68013B08495B181B041C0CEC
:1015FC00074802681B0E15684B5513689C466144DE
:10160C004C70043A026030BD2C15002004020020FE
:04161C00E0140020B6
:10162000044B1A68111D1960034B1B68043B1B68AF
:0C16300053607047E0140020E814002014
:10163C00024B1B681A68024B1A607047E8140020B2
:04164C001015002055
:10165000064B1B681A68002A04D1054A12681168F3
:10166000044A1160043B014A13607047E0140020F3
:08167000E81400201015002011
:10167800154B1B68154A19681160154A934218D909
:10168800144A1268022A07D0043B0F4A1360124A10
:101698001368013B136070470F4A11680F4A1268BC
:1016A8009142F1D10D4A002111600A4A03311160BB
:1016B800EAE7064B00221A60064B1B68022BEAD1A8
:1016C800044B03321A60E6E7E814002010150020E6
:1016D80018130020F8010020041500203C150020F4
:1016E800054B00221A605A609A6018000C300349B2
:1016F8000860DA607047C04688130020E0140020B4
:0C170800014B03221A607047F80100201A
:0C171400014B01221A607047F801002010
:0C172000014B00221A607047F801002005
:10172C0030B50D4B1C68221D1A600C490B685A1CF5
:10173C000A60587800069A1C0A609A7812040243D0
:10174C00D81C0860D87800021D1D0D601B7913434E
:10175C000343636030BDC046E01400201015002028
:10176C00054A1368191D116004490A68501C086069
:10177C0052785A607047C046E014002010150020C3
:10178C00074B19680A1D1A60064A1368581C10602A
:10179C005A781201044B9B189B684B607047C046EB
:0C17AC00E01400201015002004080020AC
:1017B800074B1A68511C19600648036851780901DB
:1017C800054A521819689160043B03607047C04687
:0C17D80010150020E01400200408002080
:1017E400074B1A68511C196051780902901C186043
:1017F40092781143802292050A431A607047C046CA
:04180400101500209B
:1018080010B5094B1868021D1A6008490B685A1C64
:101818000A605A7812029C1C0C609B781A43802339
:101828009B051343436010BDE814002010150020E9
:10183800074B1A68511C196051780902901C1860EE
:1018480092781143802292050A431A607047C04675
:041858001015002047
:10185C0010B5094B1B681A68023A80239B05134389
:10186C001A78742A03D1013B044A136010BD034A51
:10187C001360FFF7DBFFF9E7E814002010150020D8
:10188C0010B50A4B1B681B68002B0CD0084A136858
:10189C00043B1360074A136803331360034A13684D
:1018AC00043B136010BDFFF7C1FFF7E7E014002005
:0818BC00E814002010150020C3
:1018C40010B50A4B1B681B68002B0CD1084A13681F
:1018D400043B1360074A136803331360034A136815
:1018E400043B136010BDFFF7A5FFF7E7E0140020E9
:0818F400E8140020101500208B
:1018FC0010B5104B1A681100103119600E490B68A5
:10190C00180008380068D060181F006890601868CC
:10191C0050600C3B0B6009480368591C01605978F6
:10192C0009029C1C04609B78194380239B050B4384
:10193C00136110BDE8140020E014002010150020E5
:10194C00204B1B681A1F12681900083908680439E3
:10195C000968521800291ADB904210DD043B1A600A
:10196C00194B1A68511C196051780902901C1860A7
:10197C0092781143802292050A431A607047103BFB
:10198C00104A1360104A136803331360F6E7904251
:10199C0010DA043B1A600C4B1A68511C1960517810
:1019AC000902901C186092781143802292050A4318
:1019BC001A60E3E7103B034A1360034A13680333CE
:0C19CC001360DBE7E81400201015002079
:1019D800024A1368043B13607047C046E8140020AD
:1019E800024A1368103B13607047C046E814002091
:1019F80008490B681A6808480260043B0B60032A10
:101A080000D87047054A8023DB0011680B43136038
:101A1800F7E7C046E0140020581500201C150020E8
:101A280010B5044C23681878FEF76EFF2368043B52
:081A3800236010BDE014002042
:101A400010B50F4B1B68002B00D010BD2020FEF7F7
:101A50005FFF2D20FEF75CFF3E20FEF759FF44207C
:101A6000FEF756FF4220FEF753FF4720FEF750FFD8
:101A70002020FEF74DFF024B01221A60E5E7C04629
:041A8000F801002049
:101A840070B50A490A68561C0E6054783619002C41
:101A940009D00D002B685A1C2A605878FEF736FFCF
:101AA400013C002CF6D1014B1E6070BD10150020C6
:101AB40010B5114B1B68002B12D0104B1B68002B68
:101AC4000ED00F4B1B68002B15D00E4A1368191D3E
:101AD40011600D4A12785A60094B00221A600AE01C
:101AE400FFF786F90028FBD0064B1A68111D196010
:101AF400FF231840506010BDF80100201815002085
:0C1B0400C4140020E01400206C15002028
:101B100010B50E4B1B68102B08D00D4B1B681868B6
:101B2000E0231B06C2180B4B9A420CD8084B1B68CB
:101B3000186804F0A1FA2020FEF7EAFE044A1368B0
:101B4000043B136010BDFEF7CBFFF4E7C814002080
:081B5000E0140020FF0B063039
:101B580010B5064C2368186804F08AFA2020FEF7AE
:101B6800D3FE2368043B236010BDC046E014002068
:101B7800F0B587B003AA2A4B13CB13C2294B1A68B6
:101B880001929A8801AB9A805B20FEF7BDFE264B36
:101B98001B68264A0C3293420DD0244A0C329342D9
:101BA8000DD3224A0C32934216D9204C1034042506
:101BB8001E4F160024E001A804F049F80CE003A821
:101BC80004F045F8194B00221A605A609A60180010
:101BD8000C3015490860DA605D20FEF795FE20207C
:101BE800FEF792FE07B0F0BD206804F041FA20200D
:101BF800FEF78AFE01350C4B1B680434B342EBD95F
:101C0800DB1B9B10AB42E7D32020FEF77DFE084B81
:101C18001B68102BE8D02068FEF75EFFE7E7C04698
:101C2800285C0008345C0008E014002088130020B9
:041C3800C8140020AC
:101C3C00F0B5D6464F464646C0B584B001AA394BDE
:101C4C0003CB03C21B7813702020FEF75BFE364BD0
:101C5C001B68002B5BD0354D00270026C0231B05CD
:101C6C009946334B9A46304B984616E02020FEF7A7
:101C7C0049FE14E06B684A46134221D12020FEF73E
:101C8C0041FE2020FEF73EFE01360137052F34D8E9
:101C9C00103543461B68B34237D9092EE6D93000BC
:101CAC00FEF718FF3A20FEF72DFE2C00083C20789A
:101CBC000028DFD0FEF726FE0134AC42F7D1D9E77D
:101CCC0001A803F0C2FF53461B68102B11D02868E3
:101CDC00FEF700FF2020FEF715FE4020FEF712FE57
:101CEC002804000C04F0C2F92920FEF70BFE023781
:101CFC00C4E7286804F0BAF9ECE70D20FEF702FE01
:101D0C002020FEF7FFFD0027C2E7002F05D104B00D
:101D1C00E0BCBA46B146A846F0BD0D20FEF7F2FD78
:101D2C00F5E7C046005E0008001500200C080020F6
:041D3C00C8140020A7
:101D400010B5044C2368186804F02BF82368043B92
:081D5000236010BDE014002027
:101D5800F0B5C64600B582B06846214B020012CBEA
:101D680012C203F074FF0D20FEF7CEFD1D4DFA23BD
:101D78009B009846A8440026012723E0FEF7C4FDEF
:101D88000134285D0028F9D1062C05D82020FEF75B
:101D9800BBFD0134072CF9D12320FEF7B5FD38002F
:101DA80003F07FFF2020FEF7AFFD2020FEF7ACFDFB
:101DB8002020FEF7A9FD01370136052E07D008358A
:101DC800A84509D02020FEF79FFD0024D9E70D2063
:101DD800FEF79AFD0026F2E702B080BCB846F0BDD7
:081DE800845400082057000894
:101DF00070B5A2B0D34B1A6820929A8869468420A5
:101E000009180A809B796A468621521813701DAC06
:101E1000CD4B220023CB23C21BAACC4B19681B91AC
:101E2000998891809B79937119AAC94B03CB03C2FE
:101E300016AAC84B03CB03C211001A880A809B78EC
:101E40008B7013AAC44B23CB23C20FAAC34B23CB43
:101E500023C21B7813700CAAC14B03CB03C21B888F
:101E6000138009AABF4B03CB03C21B88138007AAA8
:101E7000BD4B03CB03C204AABC4B03CB03C21B78EC
:101E8000137002AABA4B19680291998891809B79C4
:101E90009371B84B01934420FEF73AFD6120FEF7A1
:101EA00037FD7420FEF734FD6120FEF731FD20A8D8
:101EB00003F0D1FEB0480C3004F082F85220FEF757
:101EC00027FD6520FEF724FD7420FEF721FD20A8E4
:101ED00003F0C1FEA94804F073F8200003F0BBFE34
:101EE000A74804F06DF85520FEF712FD7320FEF7A9
:101EF0000FFD6520FEF70CFD7220FEF709FD3D2069
:101F0000FEF706FD9F4804F05BF80D20FEF700FD8C
:101F10009D4B1B68002B00D1D6E019A803F09BFE57
:101F2000994B1B68002B00D0D2E016A803F093FE5B
:101F3000964B1B680024002B00D1D3E0914E934DAB
:101F40002B68013B1B01F318185D002804D0FEF735
:101F5000DFFC0134082CF3D113A803F07CFE8C4B7A
:101F6000186830231843C0B2FEF7D2FC0FA803F064
:101F700072FE884D884E32685101891A8B01591AB8
:101F8000C90089188901286804F0A0F80400FEF748
:101F9000A7FD2E20FEF7BCFC33685A01D21A91002F
:101FA000C918C900286804F091F863011B1B9B0045
:101FB0001B19DB00C01AFEF793FD4D20FEF7A8FCAD
:101FC0004820FEF7A5FC7A20FEF7A2FC0D20FEF7C4
:101FD0009FFC0CA803F03FFE704C2068FEF780FDCC
:101FE00023680B2B00D18AE06C4B1B68132B00D1AC
:101FF0008CE06A4B1B68262B00D18BE0674B1B687B
:10200000392B00D18AE03020FEF782FC3020FEF729
:102010007FFC634B1B68002B00D183E02020FEF780
:1020200077FC2020FEF774FC5320FEF771FC502053
:10203000FEF76EFC4920FEF76BFC3D20FEF768FCC6
:10204000584B1868FEF74CFD2C20FEF761FC564BF0
:102050001B68102B6AD0554B1868FEF741FD2C20E9
:10206000FEF756FC524B1868FEF73AFD07A803F03E
:10207000F2FD504B1B68002B00D0A1E00020FEF7C2
:102080002FFD04A803F0E7FD4B4B1868002800DA89
:10209000D4E0454B1B68102B00D1D3E0FEF720FDA8
:1020A00002A803F0D8FD454B1868002800DACCE000
:1020B0003D4B1B68102B00D1CBE0FEF711FD0D202E
:1020C000FEF726FC22B070BD1BA803F0C4FD24E778
:1020D0002320FEF71DFC2C4B18683030C0B2FEF7F1
:1020E00017FC22E76E20FEF713FC6F20FEF710FCB2
:1020F0006E20FEF70DFC6520FEF70AFC2CE735206C
:10210000FEF706FC3220FEF703FC6DE73220FEF7F7
:10211000FFFB6EE73420FEF7FBFB6FE73620FEF790
:10212000F7FB70E709A803F096FD77E71F4B1868E7
:1021300003F0A2FF2C20FEF7EBFB1D4B186803F009
:102140009BFF93E7405F0008485F0008545F00086A
:102150005C5F0008645F0008705F00087C5F000837
:102160008C5F0008985F0008A45F0008AC5F00085F
:10217000B85F00084F46460088130020181300205F
:1021800004020020040800205415002040150020FF
:102190005815002000020020DC14002068150020E3
:1021A00064150020D0140020C8140020D81400208A
:1021B000D414002014150020F8140020F41400207A
:1021C000254B1E68642575432900244803F07EFFD3
:1021D0000400FEF785FC6643B3059B1B9C01A41914
:1021E0006400A419E4001E4B9C4664442E20FEF7B4
:1021F0008FFB2900200003F069FFFEF771FC290026
:10220000200003F088FE8C00641864002900200080
:1022100003F05CFF06002900200003F07CFE88002C
:1022200040184000290003F051FF042383429B41E2
:102230005B42F6183000FEF753FC22E701A803F0DA
:102240000AFD2DE703F018FF2AE701A803F003FDBC
:1022500035E703F011FF32E730150020C0C62D002E
:0422600080C3C9016D
:1022640010B588B001A91F4B0A0013CB13C213CBBE
:1022740013C21B6813601C4A13681C68043B136078
:10228400112C17D0192C28D0382C0FD12624132C1C
:1022940014D0262C12D0392C10D0602C0ED0134A16
:1022A4008023DB0011680B43136014E0572C02D128
:1022B400392403E00B24962C10D1602401A803F0E8
:1022C400C8FC0D20FEF722FB094B1C60FDF7DCFF68
:1022D400084B00221A6008B010BD13240B2CEDD05B
:1022E400D5E7C0468C540008E01400201C150020DB
:0822F4006815002064150020AC
:1022FC0070B5FEF779FD041E00D1D7E0C0B26F4B6C
:10230C001B68002B08D06E4B1B68002B04D06D4B48
:10231C0018706D4B01221A600A2800D1C3E0022804
:10232C0000D8C2E0664B1C68002C08D109281ED0CE
:10233C00664B1B683F2B02D9202800D19DE0282832
:10234C0017D02F283FD01B2867D1002C00D1ADE02F
:10235C000E38FEF7D7FA5D4B1A685D4B2021995465
:10236C009B18002159705B4B1A6002249EE01730B9
:10237C00DEE7594B1C68002C01D0002496E0FEF7D8
:10238C00C1FAFEF731FD0028FBD0C0B220280BD0DB
:10239C004E490B684E4A2825D554D218507002333A
:1023AC000B60FEF7AFFA81E0484B1B6801334A4AD9
:1023BC0013601838FEF7A6FA2020FEF7A3FA0820BF
:1023CC00FEF7A0FA72E0444B1C68002C01D00024EC
:1023DC006CE0FEF797FAFEF707FD0028FBD0C0B2C1
:1023EC002F280BD039490B68394A2F25D554D218D0
:1023FC00507002330B60FEF785FA57E0334B1B68C5
:10240C000133354A13602738FEF77CFA2020FEF79B
:10241C0079FA0820FEF776FA48E0092848D0122805
:10242C0048D0082817D12C4B1D680024002D3DD115
:10243C00264B1C68002C39D0013C1C60244B2022FC
:10244C001A55FEF75FFA2020FEF75CFA0820FEF71B
:10245C0059FA2C002AE00D2817D11C4B1B68002BB5
:10246C000BD11A4B1A681A4B202199549B18002136
:10247C005970184B1A60012418E0174B1B68012B7C
:10248C00EFD00D20FEF73EFAEBE7134B1C68002C47
:10249C0012D10E4D0E4B2A689854FEF733FA2B6866
:1024AC0001332B6002E0002400E00024200070BD0A
:1024BC000324FBE70424F9E70024F7E7F8010020E4
:1024CC00181500206C150020C4140020B81400202E
:0C24DC00F8130020BC1400202415002080
:1024E80010B50023054A1360054A1360054A1360B6
:1024F800FFF700FF0028FBD0012010BDB814002012
:08250800BC1400202415002082
:1025100010B5154B1968154B5A5C202A09D14B1C74
:102520001248013819000133C25C202AFAD00E4B40
:1025300019600023002A10D00C4840180C4CC25CD3
:10254000202A03D01A5501330F2BF8D1084A002056
:10255000D0545B18074A136010BD054B00221A7057
:10256000044B1960F8E7C046AC140020F8130020B3
:082570005C140020B8140020E7
:10257800F0B5DE46474680B587B00E0002AA0024B3
:1025880005E0002B1BD001340132102C08D0035D6C
:102598001370190061391929F3D8203B1370F2E739
:1025A800002302AAD37313782D2B0ED1254B0022BA
:1025B8001A6001239B460127012C0FD82CE0002329
:1025C80002AAD37313782D2B2CD01E4B00221A602D
:1025D80000239B4600270120002C2DD0194B1D6895
:1025E800B84602AB9C46E044002301934346187862
:1025F800310003F0E6FB431C18D075432D18013752
:1026080001239C46E0440193A742EFD30D4B1D6084
:1026180001205B46002B0FD00A4A13685B42136007
:10262800012009E00020012CC0D105E0019B002B0E
:1026380001D0044B1D60002007B0C0BCBB46B046AB
:08264800F0BDC046B0140020F3
:1026500010B5344B187800285AD000233149013383
:102660005A5C002AFBD12D280FD0302829D12D4AC1
:10267000527820218A43582A11D02B4A11681029F8
:102680003AD1082B48D900204BE0012B3AD0264AFA
:10269000116810292AD00B2B3ED9002041E0214A95
:1026A00092782D2A09D00A2B2ED81E4810210230EC
:1026B000FFF762FF431E984133E00B2BF5D9002052
:1026C0002FE02528D9D1174A52782D2A09D00B2B73
:1026D0001CD814480A210130FFF74EFF431E9841D1
:1026E0001FE00C2BF5D900201BE000232D28C8D1BA
:1026F000092B11D9002014E02D28CCD000200A2B62
:102700000FD809E000200CE000200AE0002008E0DB
:10271000054B19681029E8D00248FFF72DFF431E2A
:0C272000984110BD5C140020C81400207B
:10272C00F0B51A4C00251A4E0021635C8A5D180026
:10273C00613819280DD8203BDBB2100061381928FC
:10274C0011D8203AD2B2934219D101310829ECD1D7
:10275C0015E01000613819280DD918002038471ED3
:10276C00B84140420340934209D1002AEDD1094BB4
:10277C001D600120F0BD203AD2B2202BE3D10135EF
:10278C0008347E2DD0D10020F4E7C046185700083D
:08279C005C140020F014002081
:1027A40070B51A4B1B78002B29D0194A00231E0040
:1027B400013310321100103909780029F7D1731C44
:1027C4001FD03301114C1C19124D16E08B4211D14C
:1027D40000290BD00132082A0CD0A15C535D1800EB
:1027E40061381928F2D8203BDBB2EFE70A4B1E60B0
:1027F400012070BD103C013E05D30022EDE700200E
:10280400F7E70020F5E70020F3E7C04604080020BE
:0C281400140800205C140020F0140020C8
:1028200010B50F4B1A680F4B1A60FFF771FEFFF7D8
:10283000B9FF002805D00C4B1B6801330B4A13600D
:1028400010BD0B4B1B78302B05D00A4A2123116891
:102850000B431360F4E7054B00221A60F0E7C04613
:10286000B8140020AC140020F01400204015002003
:082870005C1400201C1500207F
:10287800074A13680749C85401331360064A93424C
:1028880004D9064A202311680B4313607047C046D9
:102898002C15002004020020FE0500001C15002055
:1028A80010B5144B18688200134BD3581A030AD476
:1028B800124A1268002A13D19B030BD48000104BD4
:1028C800C358984705E00F4A80239B0011680B43C3
:1028D800136010BD0B4A082311680B431360F8E717
:1028E800DB0304D58000064BC3589847F1E7FFF790
:1028F800BFFFEEE7F0140020205500082015002047
:08290800000000201C15002056
:1029100070B594B00CA9414B0A0013CB13C213CB72
:1029200013C203CB03C205A93D4B0A0013CB13C24C
:1029300013CB13C21B7813706A463A4B13CB13C2E6
:1029400011001A680A601B790B71374B1B68522BF8
:1029500009D95224354E344DA05DFDF7D9FF01341D
:102960002B68A342F8D85223314A1360314A002120
:102970001160314A13602E4D304E03E02C4B1A6823
:102980002D4B1A60284C2B682268934234D2FFF7F3
:10299000BFFD3378002BF6D0FFF75AFE00280BD08E
:1029A000274B1A68274B1A60274B1B68002BE5D072
:1029B000264B01221A60E1E7FFF7B8FE002811D08C
:1029C000234B1B689B00234A9B585B0321D5FFF7D1
:1029D0006BFF214B1B68002B08D1154B1A68164B57
:1029E0001A60CFE70CA803F036F905E01A4B002275
:1029F0001A60684603F02FF90D20FDF789FF522376
:102A0000094A13600A4A13600A4B00221A6014B084
:102A100070BD05A803F01FF9EEE7C046185E000878
:102A2000385E0008545E0008BC140020F813002033
:102A3000B814002024150020AC1400205C140020E1
:102A4000B01400203415002018150020381500207F
:0C2A5000F0140020205500081C15002088
:102A5C0070B519490B681A6818480260043B0B6082
:102A6C00002A28D0164C174D174E0DE0144B00229F
:102A7C001A6020E0FFF746FF144B1B68002B1AD19D
:102A8C000E4B1B68002B16D0FDF782FB2368022B24
:102A9C00ECD02B68002BF3D03368002BF0D0FFF771
:102AAC0027FC0128E6D00228E6D1084A80235B00E7
:102ABC0011680B43136070BDE01400200815002052
:102ACC00C0140020F8010020181500201C1500204F
:102ADC0010B5044B1A68642311684B431360FFF75D
:082AEC00B7FF10BDE01400204B
:102AF40070B56E20FFF7BEFE0C4D2C68FF20FFF76B
:102B0400B9FEFF20FFF7B6FE2B68013B084A9B186D
:102B14001B04180C074909681B0E0D6853550B68F4
:102B24009C46624450700C6070BDC0462C15002059
:082B340004020020E01400205F
:102B3C0010B56F20FFF79AFE064A1368191D116035
:102B4C00054A12685A60FF20FFF790FEFF20FFF73E
:0C2B5C008DFE10BDE01400202C150020A0
:102B680010B57320FFF784FE064A1368191D11601B
:102B7800054A12685A60FF20FFF77AFEFF20FFF728
:0C2B880077FE10BDE01400202C1500208A
:102B9400F8B57420FFF76EFE104E33681D680135DA
:102BA4000F4C2D19280AFF273840FFF763FE380021
:102BB4002840FFF75FFE0B4B1B68013B1B19326873
:102BC400190A106821541268A41863707620FFF75C
:102BD40051FE3368043B3360F8BDC046E014002066
:082BE400040200202C15002062
:102BEC0010B5234B1B68002B17D1224B1B68224AB4
:102BFC0019681160214A93422ED9214A1268022A7F
:102C0C001DD0043B1B4A13601E4A1368013B136022
:102C1C001D4B1A681D4B1A6010BD6420FFF726FE71
:102C2C000022134B1A601A490B6801330B601B010D
:102C3C0018495A54184B1A68184B1A60E8E7114A8D
:102C4C001168174A12689142DBD1154A00211160B4
:102C5C000B4A03311160D4E7074B00221A60084B72
:102C6C001B68022BD4D1064B03321A60D0E7C04646
:102C7C0020150020E8140020101500201813002047
:102C8C00F801002004150020FC140020C8140020BA
:102C9C0000150020040800202C1500202815002009
:042CAC003C150020B3
:102CB00070B5324B1B68002B27D1314B1B681C7839
:102CC00023005F3B022B16D97D20FDF721FE20203B
:102CD000FDF71EFEFEF750FF25006F3D072D15D9AD
:102CE000733C012C1CD9032D0FD8264B1B68188868
:102CF00003F08CF909E0244B186801300005000D41
:102D000003F084F92920FDF703FE70BD2020FDF7B4
:102D1000FFFD5220FDF7FCFD3A20FDF7F9FDDFE74E
:102D2000184B1A68194BD31A082BEED90C3A108895
:102D300003F06CF92020FDF7EBFD2020FDF7E8FD06
:102D4000104C2368083B188803F060F92020FDF739
:102D5000DFFD6920FDF7DCFD2368043B188803F0E4
:102D600055F92020FDF7D4FD7820FDF7D1FD23682B
:102D70001888013003F04AF9C7E7C0461C15002047
:102D80000C150020E8140020101500201813002056
:102D9000084B1868084B1B68984208D001D2181AD3
:102DA0007047C01A80239B009C466044F8E70020CF
:0C2DB000F6E7C04644150020481500203E
:102DBC0010B5094B1C68221D1A60084B1B68002BB0
:102DCC0006D0074B1B68002B02D0064B186801E09D
:102DDC00FFF7D8FF606010BDE0140020F801002060
:082DEC0018150020C41400209A
:102DF40010B50B4B1C6800230A4909190A48CA5C20
:102E0400222A03D01A5401334F2BF8D1064A222127
:102E1400D15401330021D154E318044A136010BD86
:102E2400AC140020F81300205C140020B814002017
:102E34001A4B1B185A781300613B192B03D8203AFC
:102E44001300373B05E02F2A1BD91300303B092B15
:102E5400F6D80F2B18D8114A10188278110061394E
:102E6400192907D8203A373A11000F2912D8180126
:102E7400401870472F2A0AD9110030390929F4D98A
:102E8400F1E701204042F4E701204042F1E701204C
:102E94004042EEE701204042EBE7C0465C140020CC
:102EA40070B5324B1B680133314A1360FFF7A0FF42
:102EB400002600242F4A03E001360134502C0ED0A2
:102EC400A35C5C2BF8D0222BF7D12A4B00221A5595
:102ED400294B1D68002D08D1264C260032E0274AD4
:102EE400022311680B4313603EE06520FFF7C2FC28
:102EF400234A13687600A41B2249CC54013313607F
:102F040000241C4D2E0005E0FFF7B4FC0134335DB2
:102F1400002B29D0285D5C28F6D12000FFF788FF1C
:102F2400431C03D00334FFF7A5FCF0E7134A022344
:102F340011680B43136017E0FDF7E8FC0135735D7E
:102F4400002B11D0605D5C28F6D12800FFF770FFDC
:102F5400431C04D00335C0B2FDF7D8FCEFE7074AA1
:102F6400022311680B43136070BDC046B8140020DF
:102F7400AC1400205C140020201500201C15002037
:082F84002C15002004020020BE
:102F8C0070B53F4B1C6824013E4B1D682900200086
:102F9C0003F096F83C4B186080235B02984230D3C8
:102FAC00394B3A4A1A603A4B1B88DB0710D4384B22
:102FBC0000221A821A803749CA6902200243CA6168
:102FCC00354A1A836422DA621A8801210A431A806C
:102FDC002D4B1B68013B9BB22D4A13852F4B1B6855
:102FEC00002B42DB2A4A138C01210B4313842C4BFC
:102FFC001B68002B3EDB264A138C10210B431384D9
:10300C0032E0AC42CFD2224A13880125AB43138065
:10301C00002324490B6024490B60012464421F4B9C
:10302C001C609023DB051868204E30401860D9686E
:10303C003140D960D868802189010143D960118C55
:10304C00A943118416490C601868194C204018606B
:10305C00D9682140D960D868802109020143D96020
:10306C00138C10218B43138470BD138C01218B4363
:10307C001384BCE7064A138C10218B431384F3E7AB
:10308C0030150020DC14002014150020FFFF000078
:10309C00000400400010024060600000F8140020A2
:1030AC00F4140020B4140020EC140020FFCFFFFF18
:0430BC00FF3FFFFFD4
:1030C0009022D205136827490B401360264A138CBF
:1030D00001218B431384254B1B68002B22DB90219D
:1030E000C905CA681F480240CA60002B22D0632B62
:1030F0002ADC9023DB051968802292010A431A60BA
:103100001A6A1B490A401A62196A802252040A4349
:103110001A62154B1A8C01210A431A84134A126849
:103120005A6370479022D205D16880239B010B43DC
:10313000D360F6E70B000968802252010A431A6047
:103140008022D2039A61ECE7084B64221A60902334
:10315000DB051968802252010A431A6040229A61F5
:10316000DFE7C046FFCFFFFF00040040F814002057
:04317000FFFFFFF06E
:103174009022D205D36830490B40D3602F4B1B6893
:10318400002B1FDB2DD0632B3FDC9023DB051A685B
:103194002B490A401A601968802212020A431A60F5
:1031A4001A6A120112091A62196A802252050A4324
:1031B4001A62244B1A8C10210A431A841F4A12687B
:1031C4009A637047130012680A401A60D968802213
:1031D40012020A43DA601B4A138C10218B431384B6
:1031E400EFE79023DB051A6813490A401A6019684F
:1031F4008022D2010A431A60802212049A61114A81
:10320400138C10218B431384DBE70C4B64221A606C
:103214009023DB051A6808490A401A60196880225D
:10322400D2010A431A6080229A61064A138C102143
:103234008B431384C5E7C046FF3FFFFFF41400200F
:08324400FFBFFFFF0004004082
:10324C00074A13681868043B1360112806D0F02352
:10325C000340A02B01D1913B18407047B120FCE7F3
:04326C00E01400204A
:1032700070B5FFF7EBFF2D4B1B68002B26D10F28F5
:103280003ED80300083B042B21D90F281FD0284B20
:103290001B68013301D006281ED0264B1B68013362
:1032A00001D0072822D044000322A2409023DB054E
:1032B000D9689143D9601968914319601D6801224A
:1032C0001100A1402943196082409A6170BD174BDB
:1032D0008022D2001A60F9E7174A138C01218B4330
:1032E0001384134B012252421A60DCE7124A138CFA
:1032F00010218B4313840F4B012252421A60D2E7F4
:10330000B12804D0094B8022D2001A60DEE70B4BB3
:10331000DA680C218A43DA601A688A431A601A68EC
:1033200008390A431A6002229A61CFE71C1500206F
:10333000F8140020F41400200004004000040048A9
:1033400070B5FFF783FF2E4B1B68002B27D10F288A
:103350003FD80300083B042B22D90F2820D0294B4B
:103360001B68013301D006281FD0274B1B6801338F
:1033700001D0072823D044000322A2409023DB057C
:10338000D9689143D9601968914319601D68012279
:103390001100A14029431960103082409A6170BD2C
:1033A000174B8022D2001A60F9E7184A138C0121CA
:1033B0008B431384134B012252421A60DBE7134AFA
:1033C000138C10218B4313840F4B012252421A603D
:1033D000D1E7B12804D00A4B8022D2001A60DEE780
:1033E0000B4BDA680C218A43DA601A688A431A6048
:1033F0001A6808390A431A60802292029A61CEE75D
:103400001C150020F8140020F414002000040040D3
:04341000000400486C
:1034140010B5FFF719FF2B4B1B68002B23D10F2886
:103424003BD80300083B042B1ED90F281CD0264B85
:103434001B68013301D006281BD0244B1B680133C1
:1034440001D007281FD04000032282409023DB05CF
:10345400196891431960D9689143D960D9680122E8
:1034640082400A43DA6010BD164B8022D2001A60F3
:10347400F9E7174A138C01218B431384124B012261
:1034840052421A60DFE7124A138C10218B431384D3
:103494000E4B012252421A60D5E7B12804D0094BE1
:1034A4008022D2001A60DEE70A4B1A680C218A4394
:1034B4001A60DA688A43DA60DA6808390A43DA603B
:1034C400D1E7C0461C150020F8140020F414002095
:0834D400000400400004004860
:1034DC0010B5FFF7B5FE2B4B1B68002B23D10F2823
:1034EC003BD80300083B042B1ED90F281CD0264BBD
:1034FC001B68013301D006281BD0244B1B680133F9
:10350C0001D007281FD04000032282409023DB0506
:10351C00196891431960D9689143D960D96802221E
:10352C0082400A43DA6010BD164B8022D2001A602A
:10353C00F9E7174A138C01218B431384124B012298
:10354C0052421A60DFE7124A138C10218B4313840A
:10355C000E4B012252421A60D5E7B12804D0094B18
:10356C008022D2001A60DEE70A4B1A680C218A43CB
:10357C001A60DA688A43DA60DA6804390A43DA6076
:10358C00D1E7C0461C150020F8140020F4140020CC
:08359C00000400400004004897
:1035A40010B5FFF751FE264B1B68002B1ED10F28C8
:1035B40036D80300083B042B19D90F2817D0214B08
:1035C4001B68013301D0062816D01F4B1B6801333A
:1035D40001D007281AD04000032282409023DB0543
:1035E400196891431960D9689143D96010BD144B8F
:1035F4008022D2001A60F9E7144A138C01218B430C
:103604001384104B012252421A60E4E70F4A138CD0
:1036140010218B4313840C4B012252421A60DAE7C7
:10362400B12804D0064B8022D2001A60DEE7084B92
:103634001A680C218A431A60DA688A43DA60D5E78B
:103644001C150020F8140020F4140020000400408D
:043654000004004826
:1036580010B5FFF7F7FD104B1B68002B0FD10F2893
:103668000ED89023DB051B8A0122824013400B49A8
:103678000A68101D0860002B0AD00123536010BD92
:10368800074B1B8A0F2210400E3A82401340EEE788
:1036980000235360F3E7C0461C150020E014002007
:0436A80000040048D2
:1036AC0010B5144BDA6814490A40DA609969802223
:1036BC0092000A439A6102F0ACFA02F0AAFA02F004
:1036CC00A8FA02F0A6FA0D4B0022DA608021090656
:1036DC001961022159610A490A609A6801210A4359
:1036EC009A60190001220B681A42FCD002F091FA80
:1036FC0010BDC04600100240FFFDFFFF002401403A
:04370C000827014049
:103710000C4B1A6801210A431A609A6801310A4366
:103720009A60190001228B681A42FCD1064B9A69F3
:1037300006490A409A61D968802292000A43DA60F9
:103740007047C0460024014000100240FFFDFFFF0B
:10375000F0B5C64600B52C4B802252049A61FFF7A3
:10376000D7FF2A4BDA6801218A43DA609A690A4353
:103770009A619024E4052668E26890462268C02099
:1037800082432260E2688243E260E268803802435A
:10379000E2601F480022826002611E4802608127A9
:1037A000FF004760C7601C48076904252F43076175
:1037B0005D698027FF032F435F61184F3A60184D02
:1037C000FD60BFF34F8FBFF36F8F40BF20BF20BF9F
:1037D00002615A69134802405A61DA680A43DA60A2
:1037E00002F01DFAFCF76CFC0F4B104A1360104AF4
:1037F000136026604346E36002F011FA5E20FDF795
:1038000087F880BCB846F0BD0004004800100240B4
:10381000000001400004014000ED00E000140048F9
:10382000AAAAAAAAFFFFBFFF141100204815002072
:04383000441500201B
:10383400F0B589B004AA624B13CB13C21B88138062
:103844006A46604B13CB13C21B7813705E4B1B6824
:103854001C68621C18D0072C03D92300A03B072B3B
:103864001BD85A4B9B699B051ED5594B594A1A6064
:103874000F232340590003228A40072B00D99DE0DF
:103884009900554841588F46043B4F4A1360FFF74F
:103894003DFF684602F0DDF935E0504A8023DB0045
:1038A40011680B4313602EE0FFF7FEFE04A802F03C
:1038B400D0F9DAE79021C905086810430860C868A0
:1038C4009043C86001229A401300414A936204263F
:1038D400002714000425A3682B43A36023681D421A
:1038E400FCD0236CFF1802F098F9013E002EF2D1AF
:1038F400354B1B68BA081A60BB0704D5324B1A68EB
:1039040013680133136009B0F0BD9021C90508683C
:1039140010430860C8689043C860D3E79021C90584
:10392400086810430860C8689043C860CAE79021DB
:10393400C905086810430860C8689043C860C1E7B7
:103944009021C905086810430860C8689043C8609E
:10395400B8E79021C905086810430860C868904317
:10396400C860AFE71E490968013108D01D48018CC1
:103974000124A14301841A49012040420860902196
:10398400C905086810430860C8689043C86099E78F
:1039940015490968013108D01248018C1024A1434B
:1039A400018411490120404208609021C90508683A
:1039B40010430860C8689043C86083E7002381E728
:1039C400745E0008845E0008E014002000100240C9
:1039D40000240140FF070000A85400081C15002023
:0C39E400F814002000040040F41400203F
:1039F0001B4B1B68032B26D81A4B1B68043B1C2B44
:103A000021D880235B02184A12689A421BD2902365
:103A1000DB051A6815490A401A60196882225200AB
:103A20000A431A60DA6803218A43DA60DA680139E6
:103A30000A43DA600A4B1B68012B0BD99023DB0584
:103A400002229A6105E00A4A8023DB0011680B43D9
:103A5000136070479023DB05802292029A61F8E799
:103A6000D0140020D8140020D4140020F0FCFFFF54
:043A70001C15002001
:103A740010B50A4A13680A4918680860191F1160CA
:103A8400086808490860190008391160086806497F
:103A940008600C3B1360FFF7A9FF10BDE014002081
:0C3AA400D4140020D8140020D0140020FE
:103AB000F0B5DE4657464E464546E0B583B0902306
:103AC000DB051B68434A13408222520093421FD1F8
:103AD000414B1C68012C1ED99023DB0502229A6100
:103AE0003E4B1B689B461B6801933D4B19683D4B41
:103AF0001D68002201269020C00580235B039A46A2
:103B00001023994680239B02984602239C4637E067
:103B1000FFF76EFFDCE79023DB05802292029A61BB
:103B2000DEE75346836133E0012C0CD99023DB059B
:103B3000023199615B461A6003B0F0BCBB46B246E5
:103B4000A946A046F0BD9023DB058021890299613A
:103B5000F0E743468361002D2CD15200038A3340A5
:103B60001A4303E05200038A33401A4363468361D9
:103B70002B00002B02D0013B002BFCD10029D3D01D
:103B8000013933008B40019F1F42CAD04B468361ED
:103B9000002C0BD0032CDCD063468361002D09D1AF
:103BA0005200038A33401A432B0010E043468361DE
:103BB000002DD7D02B00013B002BFCD15200038AF3
:103BC00033401A43002CD1D02B00032CCED04746D3
:103BD0008761CEE70F030000D0140020E01400201E
:083BE000D8140020D4140020C9
:103BE80010B5074A1368191D1160064A12685A6011
:103BF800FF20FEF73DFEFF20FEF73AFE10BDC0464F
:083C0800E01400202C1500203F
:103C1000F8B5104E33681D6801350F4C2D19280A70
:103C2000FF273840FEF728FE38002840FEF724FE24
:103C30000A4B1B68013B1B193268190A1068215492
:103C40001268A41863707520FEF716FE3368043BF3
:103C50003360F8BDE0140020040200202C15002081
:103C600070B57D280DD8C0000E4D441908352D18AB
:103C70002078002804D0FCF74BFE0134AC42F7D189
:103C800070BD7F2528400001074D441908352D18C7
:103C900020780028F4D0FCF73BFE0134AC42F7D189
:0C3CA000EEE7C04618570008040800209A
:103CAC0070B50001064D441908352D1820780028F0
:103CBC0004D0FCF727FE0134AC42F7D170BDC046EE
:043CCC0004080020C8
:103CD000F0B5C64600B582B0AA4B1A6800929B8820
:103CE0006A469380A84B1D68002D03D002B080BCAB
:103CF000B846F0BDA54B1B68A54A13601B789846D3
:103D00001F00A44B1B685E00F6180D20FCF700FE98
:103D1000002E06D02C002020FCF7FAFD0134A6422C
:103D2000F9D19B4B188802F071F92020FCF7F0FDC7
:103D3000404602F06BF92020FCF7EAFD7E2F1AD8EE
:103D40004046FFF78DFF6A2F53D06B2F57D06C2F53
:103D500000D182E06D2F00D187E06E2F56D0702FFA
:103D600000D18AE0712F00D18DE0FD224346723BE5
:103D700013424BD059E02D20FCF7CAFD3E20FCF742
:103D8000C7FD2020FCF7C4FD4046FFF769FF7F4BCD
:103D90001B685B787F241C40682F00D19EE0692F50
:103DA00000D1A5E0642F00D1C6E07B4C032D00D1EB
:103DB000D6E02368022B00D8D2E0FCF7EFF9FEF73B
:103DC000E7FF0028F2D0FEF799FA0500012800D19C
:103DD000BCE0022800D1BCE00428E7D16D4B1B6891
:103DE000002B00D1BCE06D4A13606B4B02221A60BD
:103DF000DCE76B4B1B681B68002B07D0C7E7684BE1
:103E00001B68191F1A680B689A42C0D0684601F0F7
:103E100022FF5E4B1B68587800029B7818430130E4
:103E200002F0F4F82920FCF773FD662F35D1574BCB
:103E30001B685C782820FCF76BFD5A4B1B68102B25
:103E400027D02000FCF74CFE2920FCF761FD4F4BEA
:103E50001B685B787F241C40A1E7514B1B681A1F2D
:103E600012681B689A42D1D291E74D4B1B681A1F0A
:103E700012681B689A42C9D989E7494B1B681B68BD
:103E8000002BC3D083E7464B1B681B68002BBDD1BA
:103E90007DE7200002F0F0F8D6E7672F00D076E744
:103EA0003A4B1A6893781B04517809060B43117931
:103EB0000B43D47824021C432820FCF729FD394BFE
:103EC0001B68102B06D02000FCF70AFE2920FCF707
:103ED0001FFD67E7200002F0CFF8F7E72820FCF786
:103EE00017FD2000FFF7E2FE2920FCF711FD5CE73B
:103EF0002820FCF70DFD2000FFF7D8FE4020FCF73E
:103F000007FD240120000830274E80190004000C12
:103F100002F0B2F82320FCF7FBFC3419A068214B17
:103F20001B68102B05D0FCF7DBFD2920FCF7F0FC0B
:103F30003BE702F0A1F8F8E72020FCF7E9FC3C2081
:103F4000FCF7E6FC2D20FCF7E3FC2EE7FEF7E0FC97
:103F50002CE70D4A80235B0011680B431360C5E614
:103F60002020FCF7D5FC43465F3B022B03D8684674
:103F700001F071FEBAE67B20FCF7CAFC2020FCF7BA
:103F8000C7FCB3E6505C00081C150020101500208B
:103F90000C15002004150020F80100203C1500201D
:0C3FA000E0140020C814002004080020D9
:103FAC0010B5FFF78FFE074B1B68002B08D1064B93
:103FBC001B681B789B00054A9B589847FEF772FEBE
:103FCC0010BDC0461C15002010150020000000205C
:103FDC0010B51B4A1368013313601A4B1A68111D74
:103FEC00196019490B6853601A787F2313401B0121
:103FFC00164AD3189B680B601B787D2B0BD8144A80
:10400C001268032A04D09B00124A9B58984710BD93
:10401C00FFF7C6FFFBE70E4B1B68032B06D00E4BBE
:10402C001B68002BF3D1FFF7D3FFF0E7FFF74AFE35
:10403C00094B1B68002BEAD1FEF734FEEFE7C046B4
:10404C0004150020E814002010150020040800209E
:0C405C00F8010020000000201C150020CE
:10406800F0B587B001AA384B13CB13C211001A68F8
:104078000A601B790B71354B1B68354C354AA418FF
:10408800A3425AD2344D314E2F0038E0FFF7A2FF39
:1040980028E0FEF779FE00280CD133681B787D2BC9
:1040A8001BD82D4A1268032A14D09B002B4A9B5810
:1040B800984717E0FEF71EF9012808D00228ECD12E
:1040C800274A80235B0011680B43136035E0FEF735
:1040D8001BFCE2E7FFF766FF04E03B68032B19D0FF
:1040E800FFF778FF1E4B1B68002B26D1174B1B6868
:1040F800002B14D00133154A1360A3421DD22A683D
:10410800002AC6D11B787D2BC0D89B00134A9B5828
:104118009847E7E7FFF7D8FDFEF7C6FDE0E70E4B47
:104128001B68032B0BD00C4B01221A6000230D4A8D
:1041380013600D4A13600D4A136007B0F0BD01A863
:1041480001F085FDEFE7C046A05E000810150020CD
:1041580004020020F40D0020F801002000000020D7
:104168001C15002018150020381500200415002003
:10417800F8B5274B1C68002C2ED1264B1B6819015B
:10418800254A5218D168C022120511420AD0234A82
:104198001168081D10601B011F4AD3189B684B60EB
:1041A8002000F8BD1B011C4AD3189A681C4B1A60E2
:1041B8001C4B01221A601C4D2F681C4C2668522388
:1041C8002B6023601A4B00221A60FFF749FF2F600B
:1041D8002660184B1C68E3E70E4B186802010E4B6B
:1041E8009B18DA68C0231B0514001C401A4204D12E
:1041F80080231843FEF73CFBD2E76820FEF738FB24
:10420800044B1868FEF734FB0A4B1C68C8E7C04625
:1042180020150020F014002004080020E0140020DD
:104228001015002018150020BC140020B814002018
:08423800241500201C150020D4
:1042400070B50023384A1360384A1360384A136047
:104250001500384E0EE0384B1B68FF2B24D8662023
:10426000FEF70AFB344B1868FEF706FB304B1A6862
:104270002E4B1A60314C2B682268934230D2FEF7E5
:1042800047F93378002BF6D0FEF7E2F900281FD06B
:104290002B4B1B68002BDED12A4A1368191D1160B5
:1042A000254A12685A60E1E76720FEF7E5FA224CDA
:1042B00003202056FEF7E0FA0223E05EFEF7DCFA68
:1042C00023681812FEF7D8FA2068FEF7D5FACDE772
:1042D000FEF768FA002809D0FFF74EFF002800D04B
:1042E00070BD134B1A68114B1A60C3E7FEF71EFA34
:1042F00000280AD0FEF7D8FA134B1B68002BEFD129
:104300000B4B1A68094B1A60B4E70F4A0123116876
:104310000B4313600D4B1A680D4B1A60044B1A685F
:10432000024B1A60DCE7C04618150020AC140020D0
:10433000B81400205C140020B0140020BC1400202D
:1043400020150020E01400201C1500202815002056
:044350002C15002008
:10435400F0B5DE4657464E464546E0B593B00CA947
:10436400BA4B0A0013CB13C203CB03C21B781370DE
:1043740007AAB74B13CB13C211001A680A609A88B4
:104384008A809B798B7103AAB24B13CB13C21B880F
:104394001380B14B1A68B14B1A60FEF7B7F8FEF7F9
:1043A400FFF900280DD1FEF7BFF9002805D1AC4A6A
:1043B400012311680B43136018E10CA801F049FCB8
:1043C40014E1A54B1A68A54B1A6007A801F041FC3B
:1043D400A44D2B681801A44C001901F04BFE0D20CC
:1043E400FCF794FA2B681A01A418E168C02212059C
:1043F400080010400190114200D0FEE01B019A4ACF
:10440400D3189C68994BE41A2405240D1B5D0125DF
:10441400642B00D1D1E0954E24E00D20FCF776FA10
:10442400019D1FE0914B1A195078000202341F5D60
:1044340007432820FCF76AFA781C01F0E5FD2920DF
:10444400FCF764FA01352020FCF760FA2020FCF721
:104454005DFA0134854B1B5D642B00D1ADE0013561
:10446400072DDAD8A0190004000C01F0CDFD3A2084
:10447400FCF74CFA305DFFF7F1FB335D1A006A3A42
:104484000A2ACFD9662B1AD0672B2ED0682B4CD092
:10449400692B57D0652BD6D12220FCF737FA734B02
:1044A4001B195B789B46A31C98465B46002B7DD06A
:1044B4006E4B434499465C460F239A466BE00134A5
:1044C4002820FCF723FA6A4B1B68102B08D0674B93
:1044D400185DFCF703FB2920FCF718FA0135B2E755
:1044E400624B185D01F0C6FDF5E760480219937848
:1044F4001B04517809060B43D7783F020434025D4C
:1045040013431F432820FCF701FA594B1B68102B57
:1045140007D03800FCF7E2FA2920FCF7F7F9013557
:1045240091E7380001F0A6FDF6E701342820FCF7F6
:10453400EDF94E4B185DFFF7B7FB2920FCF7E6F9C0
:10454400013580E701342820FCF7E0F9474B1F5D73
:104554003800FFF7A9FB3F01083743483F184020C4
:10456400FCF7D4F93804000C01F084FD2920FCF791
:10457400CDF9013567E75C20FCF7C8F9380901F08B
:104584005AFB5046384001F056FB013C01239C463F
:10459400E144002C09D04B461F783B00203B5E2BA6
:1045A400E9D83800FCF7B2F9EFE7D8444446013CB7
:1045B4002220FCF7ABF9033545E72C48201800040A
:1045C400000C01F021FD3A20FCF7A0F93B20FCF798
:1045D4009DF9244B1A681201234B9B18DA68C023F7
:1045E4001B051A4209D10D20FCF790F913B0F0BC59
:1045F400BB46B246A946A046F0BD03A801F029FB7C
:104604001B4B1B68102B18D0164B1A681201164B43
:104614009B18986801F0C3FB2020FCF777F9402031
:10462400FCF774F90F4B1868000108300E4BC018E2
:104634000004000C01F01EFDD5E70A4B1A681201B4
:10464400094B9B18986801F015FDE5E7705C0008BC
:10465400885C00089C5C0008B8140020AC1400209E
:104664001C150020F014002004080020040200207F
:04467400C814002046
:10467800134B1B68134A1360134A1268120113493B
:104688005218BE20C000844661448A420AD21049AA
:104698000139891A8908013189005118002001C29D
:1046A8008A42FCD10B4A934209D80B4A9B180B4902
:1046B8008C4662440021197001339342FBD1704744
:1046C8002C150020281500200015002004080020C3
:1046D800F40D0020FE05000004020020FF05000084
:1046E80010B5164B1A68164B1A60FDF70DFFFEF74A
:1046F80055F800280DD0114B1A68114B1A60114B50
:104708001B68032B0BD8104A802311680B431360D6
:1047180004E00D4A212311680B43136010BD0B4AB6
:1047280013600B4A1B0100219954D318DB681B0541
:104738001B0D084A1360FFF79BFFEFE7B814002032
:10474800AC140020F01400201C15002000150020D7
:08475800040800202C150020CC
:1047600010B50023204A1360204A1360204A1360CA
:10477000204A1360204A1360204A01211160204A18
:104780001360204B1A68204B1A60204A00231178CE
:10479000002903D0013310325F2BF8D11C4A13607B
:1047A0001C4A1D4BD35C642B1CD01B4B1100013BDE
:1047B000CA5C642A02D0002BF9D102E0002B00D0A1
:1047C0000133164A1360FFF757FF154A154B1A605D
:1047D00000231360144A0F491160144A1360FCF758
:1047E00083FF10BD0C4BEBE72415002020150020A3
:1047F000181500203815002004150020F8010020AD
:10480000C4140020FC140020C81400200408002058
:104810000015002004020020FF0500002C150020D8
:1048200018130020E8140020101500201C1500208B
:1048300030B5B3B030AA984B1968309199889180FF
:104840009B7993712EAA954B19682E919988918026
:104850009B7993712BAA924B03CB03C211001A8848
:104860000A809B788B7028AA8E4B13CB13C225AA83
:104870008D4B03CB03C211001A880A809B788B7082
:1048800021AA8A4B13CB13C21B8813801BA9884B08
:104890000A0013CB13C203CB03C21B78137017AAF1
:1048A000844B13CB13C21B68136013AA824B13CB28
:1048B00013C21B8813800EAA804B13CB13C21100A6
:1048C0001A680A609B888B8008A97D4B0A0013CB6D
:1048D00013C203CB03C21B78137004AA794B13CB0A
:1048E00013C21B7813706A46774B13CB13C21B8815
:1048F0001380764B1A68764B60339A4200D27CE084
:1049000074490423086803430B60714B0C339A42CB
:1049100004D2704A042311680B4313606E4B1B686A
:10492000002B0FD06D4B19686D4B09010022CA5442
:104930005B185A709A70DA701A715A719A71DA713A
:104940009A60DA60644B00221A60664B1B68002B89
:104950000ED00024634D2020FBF7DAFF01342B68D2
:10496000A342F8D85E20FBF7D3FF0D20FBF7D0FF62
:1049700030A801F070F9574C206801F047FB3D204A
:10498000FBF7C6FF2368DB075AD4524B1B689B0713
:104990005AD4504B1B685B075AD44E4B1B681B07FD
:1049A0005AD44C4B1B689B065AD44A4B1B681B06B7
:1049B0005AD4484B1B68DB055AD4464B1B689B05F1
:1049C0005AD4444B1B685B055AD4424B1B681B05E9
:1049D0005AD42EA801F03FF9424B1868FCF780F832
:1049E0002920FBF795FFFFF7BBFE0D20FBF790FF9B
:1049F0003D4B00221A6033B030BD354B0C339A4228
:104A000000D286E7334B1B68002B00D086E7324B81
:104A10001B68002B3CD1354B1B68012BE5D02020B7
:104A2000FBF776FF6F20FBF773FF6B20FBF770FF40
:104A30002F4B1B68102BD8D14820FBF769FFD4E718
:104A40002BA801F008F9A0E728A801F004F9A0E7D5
:104A500025A801F000F9A0E721A801F0FCF8A0E7E3
:104A60001BA801F0F8F8A0E717A801F0F4F8A0E7F8
:104A70000EA801F0F0F8A0E713A801F0ECF8A0E709
:104A800008A801F0E8F8A0E704A801F0E4F8A0E71E
:104A9000684601F0E0F8A8E7DC5C0008E45C000888
:104AA000EC5C0008F85C0008045D0008105D00087C
:104AB000205D0008385D0008485D0008585D00086A
:104AC0006C5D0008845D0008945D0008E01400201F
:104AD000881300201C150020201500200015002040
:104AE00004080020AC1400203815002024150020F4
:044AF000C8140020C6
:104AF40010B500231E4A136001221E490A601E4994
:104B04000B601E490A601E4A5168F02081435160BF
:104B1400516851601B4A13601B4A082111601B4AEB
:104B24002A3111601A4A13601A4A1360013B1A4A67
:104B340013601A4A13601A4B312256240021C020F4
:104B440000051C705A709970D86099601033013256
:104B5400D2B2352AF5D1134B313A1A6000231049E9
:104B64003C328B54104A1360FFF7F8FD10BDC04669
:104B740054150020F801002040150020DC1400200A
:104B840000100240D0140020D8140020D4140020B7
:104B94003015002014150020F8140020F41400200F
:0C4BA40004080020001500202C15002043
:104BB00070B5164C164D2B682360FDF7A9FC2B68C9
:104BC0002360144B1D68013D28006B1C17D02D017C
:104BD000114BED18114E10E08B420BD1002913D070
:104BE0000132A95C935D1C00613C192CF4D8203B78
:104BF000DBB2F1E7103D013804D30022F1E70120D8
:104C0000404201E00120404270BDC046AC1400208B
:104C1000B814002000150020040800205C140020B7
:104C200010B5FFF7C5FF0400431C0DD002011D4B5A
:104C30009B18DA68C0231B051A420BD01A4A80233E
:104C400011680B43136010BD174A212311680B43F1
:104C50001360F8E7FFF7ACFF431C11D00201114BC2
:104C60009B18DA68C0231B051A420FD1844213D95E
:104C70000C4B24011C19A268000118188260E2E79D
:104C8000094A212311680B431360DCE7064A80239D
:104C900011680B431360D6E7034A802311680B4366
:0C4CA0001360D0E7040800201C15002061
:104CAC0010B5FFF77FFF431C0FD003010D4AD2183C
:104CBC00D3681B051B0D0C495B1892689A420AD3EA
:104CCC000001084A1018836010BD084A212311689E
:104CDC000B431360F8E7054A802311680B431360FC
:104CEC00F2E7C04604080020040200201C15002036
:104CFC00074B1A68511C196051780902901C1860F6
:104D0C0092781143802292050A431A607047C0467C
:044D1C00101500204E
:104D200010B5084B1B681B68002B08D0064A136897
:104D300002331360034A1368043B136010BDFFF78E
:0C4D4000DDFFF7E7E01400201015002054
:104D4C0010B5094B1B68191F1A680B689A4208D1D9
:104D5C00064A136802331360034A1368043B13605A
:104D6C0010BDFFF7C5FFF7E7E01400201015002079
:104D7C0010B5094B1B68191F1A680B689A4208DD9D
:104D8C00064A136802331360034A1368043B13602A
:104D9C0010BDFFF7ADFFF7E7E01400201015002061
:104DAC0010B5094B1B68191F1A680B689A4208DA70
:104DBC00064A136802331360034A1368043B1360FA
:104DCC0010BDFFF795FFF7E7E01400201015002049
:104DDC0030B589B001A80E4B020032CB32C232CBB7
:104DEC0032C21B88138000F030FFFBF7FDFF002858
:104DFC00FBD0FF231840592805D0064800F025FFAA
:104E0C00002009B030BD0D20FBF77CFD0120F8E738
:084E1C00B05D00081455000808
:104E2400F0B58FB0040001A9394B0A0023CB23C28B
:104E340023CB23C223CB23C203CB03C2354B1B6832
:104E44005F2B12D0344D354E33682B60FDF75EFB7B
:104E540033682B60FDF7FAFB051E10D0304A80231F
:104E640011680B431360002506E02D4A8023DB0004
:104E740011680B431360002528000FB0F0BDFDF747
:104E840053FC002804D10CA801002A00254F0EE091
:104E940001A800F0DEFEFFF79FFF0028F3D10225F2
:104EA400EAE7002B12D0072A0AD001320131D35D80
:104EB4000B701E00613E192EF3D8203B0B70F2E7F5
:104EC400174A022311680B431360D5E70CAB1B7818
:104ED400002B0CD00F4A1268120113495218535573
:104EE40001354378002B02D00130072DF7D1094B4F
:104EF4001A6812010C4B9B185D1900226A700B4A48
:104F040010680B4A82189A602043D8600125B3E7E1
:104F1400C854000800150020AC140020B814002068
:104F24001C1500205C140020040800202C1500200F
:044F34000402002053
:104F380070B5C0200005FFF771FF00280DD00A4C9E
:104F480022680A4803681D010949491915688D60D6
:104F5800043A22600133036070BD064A8023116859
:104F68000B431360F8E7C046E0140020001500204A
:084F7800040800201C150020B4
:104F800010B50020FFF74EFF002808D0022807D0F8
:104F9000074B1A68074B1A60074B01221A6010BDB5
:104FA000064B1B681B01064A00219954F7E7C046CF
:104FB0002C150020281500202015002000150020A9
:044FC00004080020C1
:104FC40010B51A4A13681C68043B1360022C1AD8E3
:104FD400002821D1164800F03CFE164800F039FEA6
:104FE40020003030C0B2FBF791FC002C18D02020F8
:104FF400FBF78CFC3F20FBF789FCFFF7EDFE002854
:1050040012D0200010BD0C4A8023DB0011680B4332
:10501400136001246442F4E7084800F01AFEDCE758
:10502400074800F016FEE2E70324EAE7E014002054
:10503400E05E0008F45E00081C150020105F000804
:04504400C05E000842
:1050480010B50120FFF7BAFF022800D910BD054CA2
:105058002060FBF717F92368002BF7D0FBF7B2F9AC
:08506800F4E7C04654150020D6
:1050700010B50020FFF7A6FF02280AD8074B1860DA
:10508000002807D1FFF736FDFBF7C4F8034B0022D9
:105090001A6010BDFBF75AFCFBE7C0465415002010
:1050A000074B1B68002B09D0054B00221A60054AEC
:1050B0001368191D1160044A12685A607047C0468F
:0C50C00038150020E014002034150020FA
:1050CC0010B5214B1A68214B1A60FDF71BFAFDF73E
:1050DC0063FB002821D01C4B1A681C4B1A601C4B1C
:1050EC001A6812011B4B9B18DA68C0231B051A4265
:1050FC0019D0194B1B68002B1BD1184B1B68002BAC
:10510C001AD117480368124A11680901114A52183A
:10511C0019689160043B036004E0124AA0231168F3
:10512C000B43136010BD0F4A802311680B431360AF
:10513C00F8E7FFF7AFFFE0E76920FDF797FB044BBB
:10514C001868FDF793FBEDE7B8140020AC140020B1
:10515C00F014002004080020181500202015002051
:08516C00E01400201C150020D6
:1051740010B50A4B1B68002B0DD1094A1368094965
:1051840018680860043B1360FDF7FEFEFDF796FF08
:10519400FDF7EEFF10BDFFF781FFEEE718150020C5
:0851A400E0140020301500208A
:1051AC0010B5114B1B68002B0DD1104A1368104918
:1051BC0018680860043B13600E4B1B88DB0705D591
:1051CC00FDF778FF10BDFFF765FFEEE70A4B1E22D7
:1051DC001A600A4B1968F020400000F071FF084B70
:1051EC001860FDF7CDFEEBE718150020E014002049
:1051FC00F81400200004004030150020DC140020BE
:04520C001415002055
:1052100010B5114B1B68002B0DD1104A13681049B3
:1052200018680860043B13600E4B1B88DB0705D52C
:10523000FDF7A0FF10BDFFF733FFEEE70A4B1E227C
:105240001A600A4B1968F020400000F03FFF084B3D
:105250001860FDF79BFEEBE718150020E014002016
:10526000F41400200004004030150020DC1400205D
:0452700014150020F1
:10527400F0B5C64600B588B069462B4B0A0013CB7F
:1052840013C213CB13C203CB03C2284B1B68002BDE
:1052940014D1274A13688024A40519680C43043BDD
:1052A4001360244B9C420CD9234A8023DB001168F1
:1052B4000B43136008B080BCB846F0BDFFF7EEFEA8
:1052C400E7E70D20FBF722FB684600F0C2FC200054
:1052D40000F074FE270080370F25032398460FE063
:1052E4000D20FBF713FB200000F068FE3A20FBF7CB
:1052F4000DFB300000F0D7FC00250134BC420ED079
:1053040026780135102DEBD0300000F0CCFC43465C
:105314002B40032BF1D17C20FBF7F8FAEDE70D20AD
:10532400FBF7F4FAC6E7C046F45400081815002049
:0C533400E0140020807F00201C150020E9
:1053400010B5214B1B68002B34D1204B1B681A6809
:10535000012A32D9012200241D490A60043B1B495D
:105360000B601C4B5868F0218843586059682143F2
:10537000596053019B1A99008918C900164B186887
:1053800000F0A4FE013880235B0498420DD2134A3A
:1053900050601348036A1B021B0AC02109060B4315
:1053A000036200239360073313600E4B1B68002BCE
:1053B00006D110BDFFF774FEC7E71022B024CBE77B
:1053C000FDF7E4FDF5E7C04618150020E0140020C5
:1053D000DC140020001002400002002010E000E079
:0853E00000ED00E014150020AF
:1053E800114B1A6801210A431A605A680F48024093
:1053F8005A601A680E4802401A601A680D4802403E
:105408001A605A680C4802405A60DA6A0F208243D0
:10541800DA621A6B094802401A635A6B8A435A6364
:1054280000229A607047C046001002400CB8FFF88E
:10543800FFFFF6FEFFFFFBFFFFFFC0FFACFEFFFF15
:10544800074B1B68002B00DBFEE7054A1168802329
:105458001B060B4313608369023383617047C046A0
:045468002CED00E047
:10546C0020286329323032302D323420572E5363AA
:08547C0068656D6D6572740036
:085484004B65726E656C3A0085
:10548C00416374697665206174206E65787420536D
:0C549C00797374656D20537461727400A4
:1054A800B83800080E3900082039000832390008D9
:1054B800443900085639000868390008943900084A
:1054C800205761726E3A2077696C6C206F7665722E
:1054D80072696465204B65726E656C204F50207749
:0C54E8002E73616D65206E616D65200003
:1054F400313238205352414D2062797465732073E0
:1055040074617274696E672066726F6D2030780002
:0C5514002063616E63656C6C65642000B0
:10552000000000000000000000000000000000007B
:10553000000000000000000000000000000000006B
:10554000000000000000000000000000000000005B
:10555000000000000000000000000000000000004B
:10556000000000000000000000000000000000003B
:10557000000000000000000000000000000000002B
:10558000000000000000000000000000000000001B
:10559000000000000000000000000000000000000B
:1055A00000000000000000000000000000000000FB
:1055B00000000000000000000000010000000500E5
:1055C00000000000000000000000000000000000DB
:1055D00000000000000000000000000000000100CA
:1055E00000000400000004000000000000000000B3
:1055F00000000000000000000000000000000000AB
:10560000000004000000040000000400000000008E
:10561000000000000000000000000000000000008A
:10562000000000000000000000000000000000007A
:10563000000004000000000000000500000005005C
:105640000000050000000400000004000000040049
:105650000000040000000000000001000000010044
:105660000000010000000100000003000000030032
:10567000000003000000030000000300000003001E
:10568000000003000000030000000300000003000E
:105690000000030000000300000002000000020000
:1056A00000000200000002000000020000000100F3
:1056B00000000100000008000000080000000800D1
:1056C00000000800000008000000080000000800BA
:1056D00000000800000008000000080000000800AA
:1056E000000008000000080000000800000008009A
:1056F000000008000000020000000200000001009D
:10570000000001000000000000000400000005008F
:0857100000000100000001008F
:105718004552524F5200000044524F5000000000C2
:10572800445550000000000053574150000000004D
:105738004F56455200000000524F54000000000030
:105748002D524F54000000005049434B0000000008
:10575800524F4C4C00000000494E4A45435400004B
:105768002B00000000000000312B000000000000AA
:105778002D00000000000000312D00000000000096
:1057880041425300000000005348494654000000BD
:10579800414E4400000000004F520000000000008D
:1057A800584F5200000000004E4F54000000000007
:1057B8002B2F2D00000000002A0000000000000030
:1057C8002F000000000000002A2F00000000000049
:1057D8004D4F4400000000002F4D4F4400000000D2
:1057E800425345540000000042434C520000000060
:1057F800425453540000000052414E444F4D0000A3
:105808003D3D000000000000213D000000000000B8
:105818003E000000000000003E3D000000000000C7
:105828003C00000000000000553C000000000000A3
:105838003C3D000000000000303D0000000000007A
:10584800564152434F4E000052455600000000009A
:1058580041525241590000004B45593F0000000099
:105868004B45590000000000454D49540000000018
:105878002E000000000000002E480000000000007C
:105888002E440000000000002E220000000000004E
:10589800445A0000000000004858000000000000C2
:1058A800584E4F50000000004D530000000000000B
:1058B8004453000000000000544958000000000054
:1058C80054494D4500000000534C45455000000028
:1058D800465245510000000050574D31000000006D
:1058E80050574D32000000004F48000000000000F3
:1058F8004F4C000000000000495055000000000017
:105908004950440000000000495A0000000000000F
:105918005244494E00000000524144430000000038
:10592800494E492D5350490053504900000000008A
:105938002E53000000000000465300000000000045
:105948004F5053000000000055534552000000001E
:1059580053454500000000004D454D000000000083
:10596800535400000000000052554E000000000093
:105978004E4F2D4442470000444542554700000021
:10598800464F52474554000041424F5254000000D0
:105998005245504C41434500524553544F524500DF
:1059A8004946000000000000434153450000000044
:1059B8003C434153450000003E434153450000002D
:1059C800454C5345000000005448454E0000000077
:1059D800444F000000000000554E54494C000000A0
:1059E8005748494C45000000414741494E000000D6
:1059F800464F5200000000004C4F4F50000000007E
:105A08004900000000000000434F4E5449000000C8
:105A1800425245414B0000005A425245414B00005A
:105A280052455455524E00003A0000000000000054
:105A38003B00000000000000646F53545200000057
:105A4800646F4C4954384200646F4C49540000005C
:105A5800646F56414C554500646F5245560000002E
:105A6800646F494600000000646F434153450000DD
:105A7800646F3C4341534500646F3E4341534500C6
:105A8800646F454C53450000646F444F00000000AC
:105A9800646F554E54494C00646F5748494C450053
:105AA800646F414741494E00646F464F5200000001
:105AB800646F4C4F4F50000052502D3100000000D1
:105AC80052502D34000000004155544F45584500B0
:105AD80042415544000000004C45440000000000CD
:105AE80053504545440000003F00000000000000FE
:105AF80053415645000000004C4F4144000000004F
:105B0800FEE7FEE7FEE7FEE7FEE7FEE7FEE7FEE765
:105B1800FEE7FEE7FEE7FEE7FEE7FEE7FEE7FEE755
:105B2800FEE7FEE7FEE7FEE7FEE7FEE7FEE7FEE745
:105B3800FEE7FEE7FEE7FEE7FEE7FEE7FEE7FEE735
:105B4800FEE7FEE7FEE7FEE7FEE7FEE7FEE7FEE725
:105B5800FEE703488546FFF743FC03E07047000073
:045B68000018002001
:105B6C0011488546114C20680434004201D080470E
:105B7C00F9E70F480F49091A082903DB00220260D4
:105B8C00043001600C480D49884205D0026804308D
:105B9C0003B4904703BCF7E700208646EC46002090
:105BAC000021074A9047FEE70018002034610008E6
:105BBC0070150020B8160020095E0008095E000868
:045BCC007D0C000844
:105BD00004207146084202D1EFF3088001E0EFF3A0
:0C5BE000098001490847000049540008F2
:105BEC0043466F727468204C6F77506F7765722DD7
:105BFC0034384D487A2F334D487A2C6E6F555342BA
:105C0C002D20666F722053544D333246303432207F
:025C1C00760010
:0A5C1E003323013B002BFCD170473B
:105C2800756E646572666C6F77212000202D2D2DAE
:025C380020004A
:105C3A0010B502003030C0B2392801D93732D0B29B
:065C4A00FAF761FE10BD37
:065C50002849502D3E0022
:105C560010B5441C0078002806D0FAF756FE013429
:0A5C6600631E18780028F8D110BD65
:105C700063616E277420534545204B65726E656CD9
:105C8000204F7073000000005573657248656164B1
:105C900065725F5374727563743D000056617243A0
:0A5CA0006F6E3A56616C75653D00A9
:105CAA0010B5040003061B0F18003030392801D93B
:105CBA0037331800FAF727FE0F200440200030304F
:105CCA00392800D90730FAF71EFE2020FAF71BFE02
:025CDA0010BDFB
:105CDC004572726F722300002028636F6C200000E5
:105CEC00206E6F7420666F756E6400005F53796E62
:105CFC0074617820457272005F537461636B204548
:105D0C00727200005F436F6D70696C65206F6E6C12
:105D1C00790000005F496E76616C696420436F64A2
:105D2C006520616363657373000000005F6F7574B9
:105D3C00206F6620436F6E74657874005F52756EC9
:105D4C0074696D65206F6E6C790000005F54687229
:105D5C006561642063616E63656C6C656400000052
:105D6C005F4E756D626572206F7574206F66205280
:105D7C00616E6765000000005F4469762E627920D1
:105D8C005A65726F000000002020636F6D70696CA3
:065D9C00696E672E2E0067
:0E5DA20010B5FAF79CFE2020FAF7B1FD10BDF7
:105DB00020636F6E6669726D20772E7570706572E4
:0A5DC0002063617365202759270056
:105DCA002F280FD90300303BDBB2092B08D90A2947
:105DDA000BD00300413B052B0AD83738C0B27047B5
:105DEA001800FCE701204042F9E701204042F6E7AB
:065DFA0001204042F3E726
:095E000028566172436F6E3D00EB
:0E5E0A0010B56A20FCF733FDFDF7E9FE10BD70
:105E1800203C2D6E6F742061204B65726E656C207E
:105E28004F50206E6F722061206E756D6265720032
:105E3800203C2D696E76616C696420666F72204221
:105E480061636B2D4374726C00000000203C2D527E
:0D5E5800756E74696D65204572726F720081
:0E5E660010B56B20FCF705FDFDF7BBFE10BD6F
:105E740020202841444320696E69742920000000D1
:0D5E8400202028414443206F66662920003D
:0E5E920010B56C20FCF7EFFCFDF7A5FE10BD6F
:105EA0002064656275672066696E69736865642041
:015EB00000F1
:0E5EB20010B56D20FCF7DFFCFDF795FE10BD6E
:105EC000283D456D7074792050726F6A656374293E
:015ED00000D1
:0E5ED20010B57020FCF7CFFCFDF799FE10BD57
:055EE0004C6F6164003D
:0E5EE60010B57120FCF7C5FCFDF78FFE10BD56
:0D5EF4002050726F6A656374206E6F2E007F
:0E5F020010B57220FCF7B7FCFDF781FE10BD54
:055F10005361766500FD
:105F16000A0010D00300400800E052008242FCD97B
:105F2600002000E05208934200D39B1A40418A4267
:0A5F3600F8D11900704700207047F1
:105F4000537461636B3D0000436F64655468726510
:105F500061643D00456D7074795F000050726F6A36
:105F60006563740020204155544F4558453D00005D
:105F70002020204C45446D6F64653D002020204367
:105F80005055636C6F636B3D0000000042617564A7
:105F9000526174653D0000002870656E64696E672B
:105FA000290000002020465245513D00487A2050EB
:0F5FB000574D313D000000002C50574D323D0041
:105FC00070B50400000FFFF738FE200E0F252840A3
:105FD000FFF733FE200D2840FFF72FFE200C28404E
:105FE000FFF72BFE200B2840FFF727FE200A284052
:105FF000FFF723FE20092840FFF71FFE280020405E
:0C600000FFF71BFE2020FAF783FC70BDA8
:10600C0010B50400000F16D12001000F17D120028B
:10601C00000F18D12003000F19D12004000F1AD142
:10602C002005000F1BD12006000F1CD10F20204093
:10603C00FFF7FDFD10BDFFF7FAFD2001000FFFF784
:10604C00F6FD2002000FFFF7F2FD2003000FFFF713
:10605C00EEFD2004000FFFF7EAFD2005000FFFF70F
:0C606C00E6FD2006000FFFF7E2FDDFE775
:1060780010B504003020FAF747FC7820FAF744FC02
:086088002000FFF7BFFF10BD6F
:10609000CA1751408B1A17D0C1174A4004B4484060
:1060A000411A48081A0000E052008242FCD9002040
:1060B00000E05208914200D3891A40419A42F8D137
:0C60C00004BC5040801A7047002070475C
:1060CC000A000FD00300400800E052008242FCD9C5
:1060DC00002000E05208934200D39B1A40418A42B0
:0860EC00F8D170470020704755
:1060F400CA1751408B1A19D0C11706B44840411A27
:1061040048081A0000E052008242FCD9002000E056
:106114005208914200D3891A40419A42F8D10CBCEA
:1061240053405840C01A5140891A704700207047A4
:106134005963000804020020691300006F6300081B
:106144000000002054610008040200000000000068
:106154002D0F00083D0F0008650F0008950F00087B
:10616400AD0F0008C10F0008E50F00080910000872
:1061740049100008A9100008091100082511000899
:106184003511000851110008611100087911000847
:10619400C1110008DD110008F911000815120008EA
:1061A400251200083512000851120008891200084F
:1061B400C1120008F912000839130008711300080D
:1061C400A9130008E5130008FD1300081D140008B6
:1061D400511400087514000899140008BD1400082F
:1061E400DD1400083D140008394F0008CD500008A4
:1061F40001150008BD2D0008B51A0008291A000869
:10620400111B0008591B0008411D0008A52E000899
:106214005515000875150008951500085D2A000835
:10622400DD2A0008B1150008CD1500085137000813
:1062340075510008AD510008115200087132000870
:106244004133000815340008DD340008A535000882
:106254005936000835380008753A0008B13A000884
:10626400791B0008E9160008591D00083D1C0008A8
:10627400554300087552000809170008151700084F
:1062840021170008411A0008E94600086147000880
:10629400214C0008AD4C00080B5E0008675E000846
:1062A400935E0008B35E0008F52A0008ED150008A7
:1062B4003D2B0008D35E0008E75E0008035F00087A
:1062C400692B0008952B0008211600085D180008AA
:1062D4003D1600085116000879160008814F000881
:1062E400ED2B0008851A00086D1700082D1700080B
:1062F4008D170008B9170008214D00084D4D0008FE
:106304007D4D0008AD4D0008E51700080918000888
:106314008D180008C518000839180008FD18000871
:106324004D190008D9190008E919000821280008A6
:1063340065220008F919000841530008F11D0008FE
:106344004950000871500008010000001413002097
:04635400006CDC02FB
:10635800206861680834094204D0002202700130C4
:066368000139FBD1704772
:10636E0020686168A2680C34124205D00B78037065
:0A637E0001300131013AF9D17047F6
:0400000508005B5B39
:00000001FF
